:100000000C946E030C9458220C94A6030C94A60333
:100010000C94A6030C94A6030C94A6030C94A603BC
:100020000C94A6030C94A6030C9414290C94E629B2
:100030000C94A6030C94A6030C94A6030C94A6039C
:100040000C94A6030C94F71E0C94A6030C94A60320
:100050000C94A6030C94B9240C94A6030C94A60348
:100060000C94A6030C94A6030C94A6030C94A6036C
:100070000C94A6030C94A6030C94A6030C94A6035C
:100080000C94A6030C94A6030C94A6030C94A6034C
:100090000C94A6030C94A6030C94A6030C94A6033C
:1000A0000C94A6030C94A6030C94A6033E063E06ED
:1000B0006A066A06E407CC06E407E407D706700779
:1000C00081078107532A7A2A722B7A2A722BC62A31
:1000D000E92A722B402B4F2B4A00220021002000DE
:1000E0001F001E0035002A001C00130037003600D8
:1000F00034002B0028610C00184208411200040053
:1001000029004B001B000E000D0014003300E1001D
:10011000000F2C68E2000000E000490039002E00CA
:10012000270026002500240023004D0031000F0089
:10013000150006000A0009004C002D0016001100F1
:1001400017440B4307002871E5001D0019001A0031
:10015000100005004E00380030002F000000E600BF
:100160002C78000F000000000000000000000000DC
:10017000000000000000000000000000000000007F
:10018000010000000000010000000000000001006C
:10019000000000000000000000000100010001005C
:1001A00001000000000000000000005C00000000F2
:1001B000F900000000000000DF5C0000FC00ED0022
:1001C000FB00A9000000F200F100F000EE00EF00DB
:1001D000A8000100F400F3000000FA000000AA00EB
:1001E000010000000000000000000100010001000B
:1001F00000000000000000000000000000000000FF
:1002000000000000000000000000000001000000ED
:1002100001000000000000000000010000000000DC
:1002200000000000000001000100010001000000CA
:100230000000000000000000000000004B00000073
:100240000000000000000000480052004600490085
:10025000000000004D004F00510050004A00010016
:100260000100000000004E0000000000010000003E
:1002700000000000000001000100010000006A0011
:10028000690068004500440000000000430042008F
:10029000410040003F00000001003E003D003C00E6
:1002A0003B003A00000001000000000000000000D8
:1002B000000001000100010001000000000000003A
:1002C000000000000000000000000000000000002E
:1002D000000000000000000000000000000000001E
:1002E000000000000000010000000100010000000B
:1002F00000000000000000000100000000000000FD
:1003000000000100010001000000000000000000EA
:1003100000000000005C0000000000000000000081
:100320000000DF5C0100C35CC45CCA5CC85CC65CE6
:10033000000001000000C55CCB5CC95CC75C01002B
:1003400001000100010000000000000000000000AA
:10035000000000000000000000000000000000009D
:10036000000000000000000000000000000000008D
:10037000010000000000010001000000000000007A
:10038000000000000100000000000000000001006B
:1003900001000100643214783C1E1E140A05222359
:1003A000252628292A2C2D2F3032333536383A3B52
:1003B0003D3E4042434547494A4C4E5051535557A4
:1003C000595A5C5E6062646668696B6D6F717375C3
:1003D00077797B7D7F81838587898A8C8E909294C3
:1003E00096989A9C9E9FA1A3A5A7A8AAACAEAFB1D0
:1003F000B3B4B6B8B9BBBCBEBFC1C2C3C5C6C7C91A
:10040000CACBCCCDCED0D1D2D2D3D4D5D6D7D7D8D3
:10041000D9D9DADADBDBDBDCDCDCDCDCDDDDDDDD25
:10042000DCDCDCDCDCDBDBDBDADAD9D9D8D7D7D62D
:10043000D5D4D3D2D2D1D0CECDCCCBCAC9C7C6C5E4
:10044000C3C2C1BFBEBCBBB9B8B6B4B3B1AFAEAC2A
:10045000AAA8A7A5A3A19F9E9C9A98969492908ED5
:100460008C8A89878583817F7D7B79777573716FAE
:100470006D6B6968666462605E5C5A59575553518A
:10048000504E4C4A4947454342403E3D3B3A383640
:10049000353332302F2D2C2A2928262523220000FF
:1004A000000000000000000000010204060A0F170F
:1004B000202C3A4A5D71879DB3C7DAE9F5FCFFFC51
:1004C000F5E9DAC7B39D87715D4A3A2C20170F0A08
:1004D000060402010000000000000000000000010E
:1004E00001010101010101010202020202020202F4
:1004F00002030303030303030304040404040404C6
:100500000505050505060606060607070707070889
:10051000080808090909090A0A0A0B0B0B0C0C0C3C
:100520000D0D0D0E0E0E0F0F0F10101111111212D6
:1005300013131414151516161717181819191A1A53
:100540001B1B1C1D1D1E1E1F2020212222232424B4
:10055000252626272829292A2B2C2D2D2E2F3031F0
:100560003232333435363738393A3B3C3D3E3F4002
:100570004142434445464748494A4C4D4E4F5051ED
:100580005354555658595A5B5D5E5F6162646566A7
:1005900068696B6C6D6F7072737577787A7B7D7E2E
:1005A0008082838587888A8C8E8F91939596989A7E
:1005B0009C9EA0A2A3A5A7A9ABADAFB1B3B5B7BA96
:1005C000BCBEC0C2C4C6C9CBCDCFD1D4D6D8DBDD6A
:1005D000DFE2E4E7E9EBEEF0F3F5F8FAFDFF0E03F6
:1005E00063006800690072006F006E000000120373
:1005F0004D0069006B00650020004800690078002C
:1006000000000403090409023B00020100A0FA09EA
:100610000400000103010100092111010001224031
:10062000000705810308000109040100010300001F
:100630000009211101000122490007058203200061
:10064000011201000200000008EDFE00000100019F
:1006500002000105010902A10185020901A10005AD
:100660000919012908150025019508750181020560
:1006700001093009311581257F9502750881060928
:10068000381581257F950175088106050C0A380209
:100690001581257F950175088106C0C005010906F1
:1006A000A101050719E029E7150025019508750145
:1006B00081029501750881010507190029FF1500C0
:1006C00026FF009506750881000508190129059582
:1006D0000575019102950175039101C011241FBE9A
:1006E000CFEFDAE0DEBFCDBF04B603FE18C08091C5
:1006F0008F0290919002A0919102B0919202873066
:10070000904BA740B04B59F410928F021092900278
:100710001092910210929202E0E0F8E3099511E044
:10072000A0E0B1E0E6EAF8E502C005900D92AE3532
:10073000B107D9F722E0AEE5B1E001C01D92AF38B4
:10074000B207E1F70E9418170C94512C0C9400008A
:1007500081E0089581E008950C94AA0308950C9413
:10076000AE031F93CF93DF9300D000D01F92CDB77D
:10077000DEB749835A836B833091610189819A8105
:10078000311114C0662359F0222349F00E94190A3E
:10079000182F682F89819A810E94C20903C00E9484
:1007A000ED09182F69817A81812F04C00E94190AEE
:1007B00069817A810F900F900F900F900F90DF91C9
:1007C000CF911F910C944911FC01262F408151813A
:1007D0006281738184810C94B10381E00895CF9389
:1007E000DF93EC0160E00E94E403BE01DF91CF9152
:1007F0000C94AF030C94BF120C94BB1208950E948A
:100800006C080E94FE032FEF84E39CE0215080409F
:100810009040E1F700C000000C94DF240F931F9379
:10082000CF93DF938C0161E00E94E403EC01B801F7
:100830000E94AC03882309F444C0B801CE010E9491
:1008400065218823F1F1B801CE010E94791F882328
:10085000C1F1B801CE010E94C120882391F1B801F5
:10086000CE010E94371E882361F1F801828188231E
:1008700009F1CB358DE5D807C1F050F4C115FCE581
:10088000DF0781F0CF3DDC45A9F40E947A0F19C043
:10089000CC35EDE5DE0761F0CD35DD4559F40E943C
:1008A000C30E08C00E94FF030CC00E94CC0E02C001
:1008B0000E94CF0EC801DF91CF911F910F910C9430
:1008C000A80380E0DF91CF911F910F9108950C94C0
:1008D00045240E947E040C944B2408950C946D04CE
:1008E00081E008950C9470040895CF93C82F0E945E
:1008F0006E048C2F0E947204CF9108950E9483236E
:100900000C9475040E94832390916001891721F053
:10091000809360010C9475040895CF93DF93CDB755
:10092000DEB72B970FB6F894DEBF0FBECDBF4F8357
:10093000588769877A878B8761110E940F0E9E0105
:100940002F5F3F4F86E0F90111928A95E9F785E024
:10095000FE013796D90101900D928A95E1F78981C0
:100960009A814C815D81452B31F09F3F31F491E0BC
:100970008F3F19F403C091E001C090E090FF09C0DF
:1009800049815A816B817C818D819E810E94300DCD
:1009900005C0C9010E94ED038111F2CF2B960FB65D
:1009A000F894DEBF0FBECDBFDF91CF910895FC015B
:1009B000808191810E945B0A0895CF93882309F476
:1009C0008AC0C82F8238C1F40E94832381FD83C06E
:1009D00069E380910201909103010E941D240E940D
:1009E000310E2FEF81EE94E0215080409040E1F7EE
:1009F00000C0000069E319C0833801F50E94832319
:100A000080FD69C063E580910201909103010E941D
:100A10001D240E94310E2FEF81EE94E02150804082
:100A20009040E1F700C0000063E5809102019091E1
:100A300003010E941F24CF910C94310E8438C1F41D
:100A40000E94832382FD47C067E480910201909158
:100A500003010E941D240E94310E2FEF81EE94E0CD
:100A6000215080409040E1F700C0000067E4DDCFF6
:100A70008CEF8C0F813AD0F46C2F80910201909111
:100A800003010E94E723882349F06C2F8091020123
:100A9000909103010E941F240E94310E6C2F8091BF
:100AA0000201909103010E941D24C5CF80E28C0FAA
:100AB000883048F4C77081E001C0880FCA95EAF712
:100AC0000E94F20DB8CFCD3E30F08C2F0E949D17C2
:100AD000CF910C946F18CF910895882309F464C0C6
:100AE000823879F40E94832381FF5EC069E380919C
:100AF0000201909103010E941D240E94310E69E3BE
:100B000010C08338B1F40E94832380FF4DC063E599
:100B100080910201909103010E941D240E94310ED8
:100B200063E580910201909103010E941F240C94BF
:100B3000310E843879F40E94832382FF35C067E444
:100B400080910201909103010E941D240E94310EA8
:100B500067E4E7CF9CEF980F913A10F4682FE1CF4C
:100B600090E2980F983050F4877091E001C0990F8F
:100B70008A95EAF7892F0E94F80DD9CF9BE5980F47
:100B8000933020F480E090E00C94AF2398E5980F28
:100B9000973120F480E090E00C94C5238D3E20F046
:100BA0000E94F8170C946F1808951F93CF93DF934A
:100BB000182FEB010E94DD04209741F08FE99FE0A0
:100BC0000197F1F700C000002197F6CF812FDF9148
:100BD000CF911F910C946D05893319F060E070E09E
:100BE00002C060E570E00C94D505882321F00E94D6
:100BF000F20D0C94310E0895882321F00E94F80D17
:100C00000C94310E0895CF92DF92EF92FF920F93E2
:100C10001F93CF93DF937C01D62FC72FFC01128146
:100C2000058102950F700E94E80D8823B9F0112309
:100C3000A9F08C2F807F803421F080E28D0F8830E6
:100C400068F080915C0282FD09C082E00E94910EF2
:100C50000E94E80D91E0D82ED92601C0D12CCC2ECF
:100C6000C2948FE0C8228C2D90E08C30910508F062
:100C7000ABC1FC01EA5AFF4F0C94E02B8C2F807F14
:100C8000CF70882311F0C295C07F112399F0CC2337
:100C900009F486C180E28D0F883010F0D11104C0B4
:100CA0008C2F0E94F20D03C08C2F0E94020E0E9416
:100CB000310E76C18D2F0E946D05CC2309F484C1BD
:100CC00080E28D0F883038F1DD2329F18C2F0E94CE
:100CD000080E24C08C2F807FCF70803211F0C29517
:100CE000C07FDD2319F0D130A1F140C080915C02BA
:100CF00082FF17C0112349F0CC2329F08C2F0E94CA
:100D0000F20D0E94310E80E04CC180E00E946D0522
:100D1000CC2309F459C18C2F0E94F80D0E94310E8A
:100D200053C1112371F0002341F0013031F40E94CE
:100D3000120E8C2B0E941A0E47C10E94120E8C2B91
:100D40000EC0002319F0013009F43EC10E94270EA5
:100D50001FC0112339F0063008F036C18C2F0E94D5
:100D6000F50532C1053008F02FC112C0112319F06A
:100D70000023A1F315C1002359F0D93309F021C193
:100D8000FFEF07EE13E0F15000401040E1F717C10C
:100D90008C2F0E94FC0518C18D2F112319F00E9481
:100DA0009D1702C00E94F8170E946F1815C18C2F62
:100DB000837009F047C011110BC12D2F2295269584
:100DC0002770220F220F6D2F6F70862F90E0A0E00A
:100DD000B0E0022E04C0880F991FAA1FBB1F0A94FF
:100DE000D2F7D4FF10C04FE050E060E070E004C0E4
:100DF000440F551F661F771F2A95D2F740955095CF
:100E00006095709503C040E050E0BA01C695C69564
:100E1000C3708A019B01082B192B2A2B3B2BC9017C
:100E2000B801C23049F058F4C13019F00E94D80816
:100E3000CFC00E94C608CCC00E94EA08C9C00E9468
:100E4000C408C6C0112319F08C2F817001C086958B
:100E5000882309F4BDC02D2F229526952770220FD7
:100E6000220F6D2F6F70862F90E0A0E0B0E0022E71
:100E700004C0880F991FAA1FBB1F0A94D2F7D4FF82
:100E800010C04FE050E060E070E004C0440F551F18
:100E9000661F771F2A95D2F74095509560957095FB
:100EA00003C040E050E0BA01C695C695C3708A0100
:100EB0009B01082B192B2A2B3B2BC901B801C230EF
:100EC00049F058F4C13019F00E949D0981C00E9478
:100ED0008B097EC00E94AF097BC00E94FE0878C0CB
:100EE000CF70112339F08C2F0E9424098D2F0E947E
:100EF000F5056EC08D2F0E94FC058C2F0E944509C0
:100F000067C0D23F21F128F4D03F41F0D13FC1F07A
:100F100043C0D33F19F1D43F79F03EC0112341F0D3
:100F2000053008F051C08C2F8F710E946A094CC0A7
:100F3000063008F049C0F7CF80915C0282FF18C0EC
:100F4000112339F08C2F8F710E9424093DC0112389
:100F5000C9F38C2F8F710E94450936C0112329F0E7
:100F60008C2F8F710E940F092FC00E940A092CC07C
:100F7000112349F0CF718C2F0E94240963E08C2F3C
:100F80000E94760E21C081E00E94910E0230E0F0B6
:100F900082E00E94910E18C0112331F0002391F2DB
:100FA0008D2F0E94DD0410C0002399F2D93349F43B
:100FB0001FEF27EE33E0115020403040E1F700C032
:100FC00000008D2F0E946D0588EF8C0D843020F479
:100FD0000E9483230E947504DD20C9F00E94E40D65
:100FE00080FD15C0F70112820E94DE0D0E942409C7
:100FF000C7010E9428080E94DE0DDF91CF911F914A
:101000000F91FF90EF90DF90CF900C944509DF9106
:10101000CF911F910F91FF90EF90DF90CF900895A7
:101020000F931F93CF93DF93EC01688179818A81BD
:101030000E94660A8C010E94C1090E94B208B80190
:10104000CE010E940306DF91CF911F910F91089569
:10105000CF93DF93EC01988189812B813C81232BF5
:1010600031F08F3F31F481E09F3F19F403C081E0FC
:1010700001C080E080FD1DC0CE010E940E048111E0
:1010800010C00E94E80D8823A1F08A81882389F08E
:1010900080915C0282FD0DC082E0DF91CF910C94C3
:1010A000910ECE010E941008CE01DF91CF910C94D9
:1010B000EF03DF91CF9108950E940F0E0E94310E31
:1010C0000E94A0190C946F18809102019091030165
:1010D0000E9421240C945C080E94FF0D0C9464086B
:1010E00092959F70963079F010F4925001C09A500A
:1010F000923068F4803F69F018F4883E40F409C0EB
:10110000843F29F406C0883E20F0813F11F080E042
:10111000089581E00895FC01808191810E945B0A1D
:101120000E9470080895CF93DF9300D000D01F92E3
:10113000CDB7DEB70F900F900F900F900F90DF910B
:10114000CF910895CF93DF9300D000D000D0CDB7DA
:10115000DEB726960FB6F894DEBF0FBECDBFDF9187
:10116000CF910895089508950C94B3080C94B40891
:101170000E94B60860939301709394018093950147
:10118000909396010C945C080C94B8080F931F93ED
:101190000091930110919401209195013091960155
:1011A000602B712B822B932B1F910F910C94B808FD
:1011B0000F931F9300919301109194012091950139
:1011C0003091960160237123822393231F910F9105
:1011D0000C94B8080F931F93009193011091940100
:1011E00020919501309196016027712782279327DE
:1011F0001F910F910C94B8080C94B3080E94FC083E
:1012000060938F017093900180939101909392016C
:101210000C945C0860E070E0CB010C94FE080F9326
:101220001F9341E050E060E070E08A019B0104C040
:10123000000F111F221F331F8A95D2F7C901B80171
:101240001F910F910C94FE080F931F9341E050E003
:1012500060E070E004C0440F551F661F771F8A9539
:10126000D2F780918F0190919001A0919101B0915E
:1012700092018A019B01082B192B2A2B3B2BC901B8
:10128000B8011F910F910C94FE080F931F9341E03A
:1012900050E060E070E004C0440F551F661F771FE8
:1012A0008A95D2F7409550956095709580918F0101
:1012B00090919001A0919101B09192018A019B01BE
:1012C000082319232A233B23C901B8011F910F9139
:1012D0000C94FE080F931F9341E050E060E070E033
:1012E00004C0440F551F661F771F8A95D2F780915F
:1012F0008F0190919001A0919101B09192018A018A
:101300009B01082719272A273B27C901B8011F91EC
:101310000F910C94FE080F931F9300918F01109171
:1013200090012091910130919201602B712B822BC1
:10133000932B1F910F910C94FE080F931F93009114
:101340008F011091900120919101309192016023C1
:101350007123822393231F910F910C94FE080F9306
:101360001F9300918F011091900120919101309174
:10137000920160277127822793271F910F910C9468
:10138000FE08089527E0929F800D1124E82FE6952E
:10139000E695E695877051E001C0550F8A95EAF70A
:1013A00085E0E89FF0011124EE59FE4F20E030E087
:1013B00070E04081CB01022E02C0969587950A9479
:1013C000E2F78170819584278523842781932F5F9D
:1013D0003F4F2530310569F7089527E0929F800D32
:1013E0001124682F669566956695982F977085E00D
:1013F000689FB001112440E050E080E0FB01E40F61
:10140000F51FEE59FE4F208130E0092E02C03695BF
:1014100027950A94E2F721703327042E01C0220F8A
:101420000A94EAF7822B4F5F5F4F4530510531F741
:101430000895BF92CF92DF92EF92FF920F931F9386
:10144000CF93DF938C01C0908F01D0909001E090FA
:101450009101F09092018091930190919401A0915B
:101460009501B0919601C82AD92AEA2AFB2ACFE130
:10147000D0E0D701C6010C2E04C0B695A79597956C
:1014800087950A94D2F780FD04C0219790F7B12C7C
:1014900007C0BC2EB8018C2F0E945C110197A9F3E4
:1014A0008B2DDF91CF911F910F91FF90EF90DF90E7
:1014B000CF90BF900895CF93DF93EC010E94190A5B
:1014C000BE010E945C11DF91CF9108951F93CF93CD
:1014D000DF93EB0190916101992321F0CB010E94F0
:1014E0005B0A13C0882349F0CB010E94190A182F08
:1014F000682FCE010E94C20904C0CB010E94ED09F1
:10150000182FBE01812F0E945C11DF91CF911F9196
:1015100008951F93CF93DF93C091970116E08091B8
:101520009801C81799F0D0E01C9FF0011D9FF00DA5
:101530001124E756FE4F408151816281738184817D
:1015400095810E94A2082196C770E9CFDF91CF91C3
:101550001F9108954091C9015091CA016091CB013A
:101560007091CC018091CD019091CE010C94A20894
:10157000209197019091980156E02917A9F030E049
:10158000529FF001539FF00D1124E756FE4F7181D9
:10159000761306C07081781303C07281741306C07D
:1015A0002F5F3F4F2770E9CF80E0089581E00895D5
:1015B000EF92FF920F931F93CF93DF938091CE0111
:1015C00082958F7009F065C08091CB01882309F462
:1015D00060C080919701F09098011091C90100912D
:1015E000CA016091CC017091CD0191E01F3F09F0DB
:1015F00090E0C0910001D0910101292F96E0E92EE1
:101600008F1509F446C06115710521F00F3F21F0D7
:1016100030E003C031E001C0322F90E030FD36C031
:10162000E89EF001E99EF00D1124DF01A756BE4FA0
:1016300011963C911197301329C03C91311326C06B
:1016400012963C911297311121C013964D915C91E5
:101650001497461B570B4C175D07C0F48091CE01C1
:101660008F7080618093CE01E256FE4F80818F7033
:101670008061808389EC91E00E942808DF91CF91FE
:101680001F910F91FF90EF900C94890A019687703B
:10169000B7CFDF91CF911F910F91FF90EF900895F9
:1016A0008F929F92AF92BF92CF92DF92EF92FF9272
:1016B0000F931F93CF93DF93CDB7DEB761970FB62C
:1016C000F894DEBF0FBECDBF8C0185E0F801DE01CE
:1016D0001D9601900D928A95E1F7D8011296EC9033
:1016E0009091C9012091CA014091CC015091CD0146
:1016F0004115510531F02F3F31F481E09F3F19F43E
:1017000003C081E001C080E080FD7CC1F801C080A1
:10171000D1808380948089ECA82E81E0B82EF0904F
:10172000CB01B401641B750B409100015091010184
:10173000FF2009F411C18091CE01382F307F64174A
:10174000750708F0CBC031118AC0D21214C0C9127B
:1017500012C0FE2CE1100FC08F7080618093CE010B
:101760000E94AA0AC5010E9428088091CE01D801D2
:1017700015968C9361C18114910439F0BFEFDB128F
:1017800006C081E0CB1203C003C081E001C080E04D
:1017900080FD03C081E08E2502C080E090E080FFE4
:1017A00010C04E2D6D2D8C2D0E94B80A882349F053
:1017B00089EC91E00E942808E9ECF1E086E0DF0185
:1017C0009DC0892839F0BFEFDB1206C081E0CB1243
:1017D00003C003C081E001C080E080FD03C081E060
:1017E0008E2502C080E090E0E82FE170BE2E80FFE1
:1017F0002CC04E2D6D2D8C2D0E94B80AF82E811113
:1018000024C0CD86DE868D859E850E945B0A292FA9
:1018100022952F70223018F0243090F405C09F706C
:1018200059F0811109C008C19F7031F0D801159697
:101830009C91907F09F400C1805E883008F4FCC060
:10184000C8010E942808FB2CF7C0FE2CEE2009F4EA
:10185000F3C08091CE0181608093CE0154C0D2123A
:1018600006C0C91204C0E11002C0F80199C0C80145
:101870000E948B08882361F1EE2051F12091CE0166
:10188000822F82958F7090E0029774F08091C90149
:101890009091CA0198878F8319869B868A862C87A8
:1018A000CE0107960E94280886E0F801A9ECB1E075
:1018B00001900D928A95E1F70E94D80A0E94AA0A27
:1018C0000AC0D21611F1C8010E948B0881112CC0E8
:1018D000C8010E942808FF24F394AEC03111F1CF53
:1018E000782D998A888AA6016E2D89890E9493088D
:1018F00089EC91E00E94280886E0D5011D928A9526
:10190000E9F70E94AA0AF12C97C0C912DCCFE110B6
:10191000DACFF8018583C8010E94280886E0D50146
:101920001D928A95E9F788C0EE2091F22091CE01B0
:10193000822F82958F7090E002970CF4B5CF809142
:10194000C9019091CA019A8389831B829D828C82EE
:101950002E83CE010196A6CF6417750708F044C008
:10196000FE2CEE2009F4B4CFD21230C0C9122EC022
:101970002091CE0120FD21C0822F82958F70482FAB
:1019800050E041155105C9F0F80125834F3051054C
:1019900041F08F5F982F9295907F822F8F70892BC7
:1019A0008583C8010E94280886E0F801A9ECB1E00F
:1019B00001900D928A95E1F73DC086E0F801A9EC0F
:1019C000B1E001900D928A95E1F736C0C8010E94FE
:1019D0008B08811169CF8091CE0181608093CE0107
:1019E000C8010E94280828C0782D998A888AA601F3
:1019F0006E2D89890E94930886E0D5011D928A95F3
:101A0000E9F718C0EE2009F463CFC8010E948B08E3
:101A1000F82E882309F45CCF86E0F801A9ECB1E048
:101A200001900D928A95E1F789EC91E00E94D7042C
:101A30000E94D80A0E94AA0A8F2D61960FB6F894C8
:101A4000DEBF0FBECDBFDF91CF911F910F91FF90F1
:101A5000EF90DF90CF90BF90AF909F908F900895C0
:101A60001F93CF93DF93CDB7DEB72C970FB6F894C3
:101A7000DEBF0FBECDBF4F83588769877A878B87BC
:101A80009C87CE0107960E94500B8823D1F09F813E
:101A900088852A853B85232B31F08F3F31F481E007
:101AA0009F3F19F403C081E001C080E080FD47C082
:101AB0004F81588569857A858B859C850E94A2080F
:101AC0003EC086E0FE013796DE01119601900D9230
:101AD0008A95E1F7FF81E8856A857B856115710547
:101AE00031F0EF3F31F481E0FF3F19F403C081E0B2
:101AF00001C080E080FD23C02091980130E0C90141
:101B00000196877099274091970150E084179507B7
:101B1000F1F1F983EA837D836C8396E0929FD00193
:101B2000939FB00D1124A756BE4FFE013196019030
:101B30000D929A95E1F7809398010E94890A16E028
:101B40008091970190919801891771F1189FC001B8
:101B5000112487569E4F0E94500B882329F1E09153
:101B600097011E9FF0011124E756FE4F40815181DD
:101B700062817381848195810E94A208809197017E
:101B800090E001968770992780939701D9CF0E94A2
:101B90006C081092980110929701E9ECF1E086E050
:101BA000DF011D928A95E9F72C960FB6F894DEBFF7
:101BB0000FBECDBFDF91CF911F9108958091D701C6
:101BC00085958595859508958091D70187700895AD
:101BD0009091D701977081E009F480E00895809199
:101BE000E20108959091E201892B8093E20108952A
:101BF00080959091E20189238093E20108951092EB
:101C0000E20108959091E101892B8093E10108950B
:101C100080959091E10189238093E10108951092CC
:101C2000E10108958091D801089508950C94150E4E
:101C30000C94160E90915C0292FD08C09091D80110
:101C4000981721F08093D8010C94180E0895809174
:101C5000D801882329F01092D80180E00C94180E46
:101C60000895CF93DF93E0910201F09103018091F9
:101C7000E2018083E0910201F09103019081809163
:101C8000E101892B80838091D801882381F0E09144
:101C90000201F09103019081892B808380910201E0
:101CA000909103010E94DB2381110E94270EC091B5
:101CB0000201D091030148E050E06FEC71E0CE01E9
:101CC0000E94F32B892B69F088E0FE01AFECB1E0B4
:101CD00001900D928A95E1F7CE01DF91CF910C949E
:101CE0009623DF91CF9108950C94150E90915C028C
:101CF00092FD10C098E0899F90011124262B20931B
:101D0000D7010E9424098091D701859585958595F5
:101D10000C94740E0C9424091092D70180E00C945A
:101D2000740E2091D701809582238093D701982F3C
:101D3000977099F430E0482F082E000C550B2417AB
:101D4000350759F090915C0292FD07C08595859505
:101D500085950E9445090C948C0E089590915C0223
:101D600092FB222720F9281769F080FB92F99093C3
:101D70005C0280915B0290915C020E94F60E82E010
:101D80000C94910E089580915C0282FB882780F963
:101D900091E089270C94AE0E81E00C94AE0E80E0A9
:101DA0000C94AE0E80E090E00E94172C21E0893E5A
:101DB0009E4F09F020E0822F089582E090E00C947D
:101DC000092C83E090E00C94092CCF9384E090E000
:101DD0000E94092CC82F82E290E00E94092C2C2F2F
:101DE00030E0A901582BCA01CF910895CF93C92F94
:101DF000682F84E090E00E941D2C6C2F82E290E01E
:101E0000CF910C941D2CAB01BC018FE090E00C94A1
:101E10002F2CAB01BC0183E190E00C942F2C60E0EF
:101E200070E0CB010C94090F60E070E0CB010E94E0
:101E3000030F0C940F0F69EE7EEF80E090E00E949C
:101E40003B2C60E082E090E00E941D2C60E083E08B
:101E500090E00E941D2C1092930110929401109218
:101E600095011092960160E084E090E00E941D2CA4
:101E700060E082E290E00E941D2C60E085E090E04E
:101E80000E941D2C60E086E090E00E941D2C6FEF08
:101E900087E090E00E941D2C40E050E0BA0188E00D
:101EA00090E00E942F2C60E08DE090E00E941D2CBD
:101EB00040E050E0BA0188E190E00E942F2C60E001
:101EC00087E190E00E941D2C40E050E0BA018CE1D7
:101ED00090E00E942F2C60E070E080E290E00E9491
:101EE0003B2C40E050E0BA0188E190E00E942F2CAA
:101EF0000C94140F0C941B0F682F8EE090E00C9440
:101F00001D2C0E9482246093F1017093F201809352
:101F1000F3019093F4016093ED017093EE018093CF
:101F2000EF019093F001089585B7806885BF85B76C
:101F3000806885BF08950C947A1408950C949D0FC1
:101F40000C949D0F0C94A00F0C949D0F0C94A40F57
:101F50000C949D0F0E94940F82E892E10E947923D5
:101F60000E94A80F0C94A60F0E949E0F0C949D0F28
:101F70000E9485120C9474040E946D240E943812F1
:101F80000E9492140E94C4130E94B80F0E94611F05
:101F90000E94551D0E94D91E0E94A6140C94A20FE7
:101FA0008F929F92AF92BF92CF92DF92EF92FF9269
:101FB0000F931F93CF93DF93CDB7DEB72A970FB65A
:101FC000F894DEBF0FBECDBF0E94E813982E81119A
:101FD0000E94810F83EEA82E81E0B82E00E010E071
:101FE000802E802F0E94A912D82EF501C1905F018A
:101FF000C826B1F40F5F1F4F0A30110589F78FEF24
:1020000089838A831B820E9476248160782F9D8336
:102010008C8349815A816B818D810E948D042FC0F0
:102020008091F50181FD0E94AF12E12CFF24F39411
:102030008C2D8F21F1F00E949B0F882399F0EE8266
:102040008F82DF2081E009F480E088870E94762477
:102050008160782F9A8789874E815F8168858A851C
:102060000E948D04F801ED51FE4F8081F826F08228
:1020700006C0E394FF0CF7E0EF12DACFBBCF81E0AC
:10208000911001C080E02A960FB6F894DEBF0FBE13
:10209000CDBFDF91CF911F910F91FF90EF90DF9017
:1020A000CF90BF90AF909F908F9008950E94D00FD7
:1020B0000E947A140E948D1D0E948D180C94820437
:1020C000CF93DF930E946111EC01811522E5920705
:1020D00078F5811531E5930708F09DC08F3F910594
:1020E00009F0B8F48D3E910508F06FC0853A91056E
:1020F00050F48430910508F0C8C0019709F0C2C0BF
:1021000081E090E0C3C0805E9109089708F4BDC0EB
:10211000B9C0811540E5940708F05DC08115904471
:1021200008F055C0C11580E2D80708F4AEC0AAC0B7
:10213000811526E5920728F5811535E5930708F006
:1021400087C0811544E5940708F07CC0AC0143705A
:102150005527282F26952695C115D34508F061C02F
:1021600081E090E002C0880F991F4A95E2F740E2B3
:10217000249F90011124EC01C22BD32BCE019C682B
:1021800085C081152AE5920780F4811539E593070A
:1021900008F067C0811548E5940708F473C0D82F8C
:1021A000CC27CE01806F906A71C090568115904205
:1021B00008F068C08D2F8F710E94F511DD27D06265
:1021C0008F71AE01582BCA0161C090655FC0DF708E
:1021D000CE01906A5BC074E0969587957A95E1F799
:1021E000282F23703C2F337081E090E002C0880FCD
:1021F000991F3A95E2F79C68AC01522B9A019C2FEB
:102200009F709695969550E2959FE0011124C90123
:102210008C2B9D2B3BC0D82FCC27CE01816F906A91
:1022200035C081E090E002C0880F991F4A95E2F71F
:1022300050E2259F90011124EC01C22BD32BCE013B
:102240009A6824C0D82FCC27CE01846F906A1EC014
:102250000E94F5118F7190E0D82FCC27CE019062AB
:1022600015C08F700E94F51194E0D695C7959A9588
:10227000E1F7CF70D0E0DC2FCC27D0699E01282B6E
:10228000C90104C080E090E001C0CE01DF91CF9190
:10229000089526E4829FC0011124FC0127E0729F6B
:1022A000E00DF11D1124E60FF11DEE0FFF1FE852A6
:1022B000FF4F8591949108950E9449110E946010EA
:1022C00008958238910569F1B0F48133910509F4DC
:1022D0006DC048F48932910509F463C08A329105D2
:1022E00009F469C008958533910509F455C089330F
:1022F0009105B9F00895833E910569F138F4803E67
:102300009105B1F0823E910509F10895863E91054F
:10231000A9F1873E9105B9F1843E910509F064C0A9
:1023200023C020915B0220FD4FC021FD4DC00895C8
:1023300080915B0280FD44C080915C0280FF44C0BC
:1023400080915B0284FD42C083EE4DC080915B02B0
:1023500082FF38C0F5CF80915B0282FD33C080914F
:102360005C0280FD31C0ECCF80915C0281FF32C005
:1023700080915B0284FD2AC087EE35C080915B02AC
:1023800083FF26C0F5CF80915B0283FD21C0809141
:102390005C0281FD1FC0ECCF80915B0285FD1CC0FB
:1023A0001DC080915B0285FD19C016C080915B0243
:1023B00086FD16C017C080915B0286FD13C010C059
:1023C00089E311C082EE0FC080EE0DC080E00BC02B
:1023D00086EE09C084EE07C089E205C085E303C02C
:1023E0008AE201C081E390E0089590915B0292FF40
:1023F0000DC0282F2871283019F4877F846006C00B
:10240000282F2471243011F48B7F886093FF0DC036
:10241000282F2871283119F4877E846106C0282F5F
:102420002471243111F48B7E886120915C0220FF9D
:102430000DC0382F3871383019F4877F816006C09D
:10244000382F3171313011F48E7F886021FF0DC03B
:10245000282F2871283119F4877E816106C0282F22
:102460002171213111F48E7E886194FD877E08955B
:1024700010925702109258021092590210925A026A
:102480000895CF92DF92EF92FF926B017C010E9440
:102490007A1481110EC00E948224C61AD70AE80A53
:1024A000F90AC0925702D0925802E0925902F09273
:1024B0005A02FF90EF90DF90CF9008950F931F93F3
:1024C0000E947A14882321F01F910F910C9482248A
:1024D0000E948224009157021091580220915902C3
:1024E00030915A02600F711F821F931F1F910F912D
:1024F00008950E947A1481110C9476240E945E1231
:10250000CB01089580E0089508950E94D20E8111B4
:1025100002C00E947A0F0E94DD0E8093F5010E9496
:10252000E50E90935C0280935B020E9484120E94ED
:10253000E10E682F70E080E090E00E94C408609196
:102540008F017091900180919101909192010C9472
:10255000FC08E82FF0E0E859FD4F808108950895C8
:1025600080EA8A95F1F7089500C008950C94B0129E
:1025700008950C94B8120C94B9120C94B8120C94DF
:10258000BD120C94B812FF920F931F93CF93DF9359
:1025900000D000D01F92CDB7DEB70E947A146091B0
:1025A00072028823E9F185E0F82E8E010F5F1F4F3C
:1025B000F8018F2D11928A95E9F7862F90E0B801E6
:1025C00088599D4F0E94B414882389F080915D0240
:1025D00090E045E050E0B80188599D4F0E94F32BF0
:1025E00021E02093F601892B61F410E016C0809160
:1025F000F6018823D1F3F8011192FA94E9F71092C9
:10260000F601A0915D02B0E0A859BD4F85E0F80148
:1026100001900D928A95E1F711E00E94FC030DC034
:1026200070E068597D4F80915D0290E088599D4F20
:102630000E943E150E94C11210E0812F0F900F9052
:102640000F900F900F90DF91CF911F910F91FF90FE
:102650000895F894E82FE295EF70F0E031A1282F6B
:102660002F7081E090E001C0880F2A95EAF7982F3B
:102670009095932391A392A1892B82A37894089596
:102680000F931F93CF93DF93C7E4D1E089918F3FDE
:1026900011F00E94291381E0CC34D807B9F7C0E4C7
:1026A000D1E007E411E089918F3F11F00E942913D6
:1026B0000C171D07C1F7DF91CF911F910F9108955E
:1026C000CF92DF92EF92FF920F931F93CF93DF93FE
:1026D0008C01C62FD0E0CE01895B9E4F7C01FC01AE
:1026E00090819F3F09F447C0D62EF894E92FE295D8
:1026F000EF70F0E081A19F7021E030E001C0220F77
:102700009A95EAF7822B81A382A12095282322A300
:1027100078940E94B412E0E4F1E047E451E031E043
:10272000C12C21912F3F89F0A22FA295AF70B0E06C
:1027300090968C9190E02F7002C0959587952A9580
:10274000E2F780FD02C0832F01C080E0C82A330F6A
:102750004E175F0731F7F70180818F3F11F00E941C
:10276000291361E0C11001C060E08D2D0E94B612F6
:10277000C00FD11FC882DF91CF911F910F91FF90A1
:10278000EF90DF90CF900895809104018091040133
:10279000811102C095E001C090E09093720285E043
:1027A000891B80935D020E9440138AE0E8E6F2E014
:1027B000DF01982F1D929A95E9F7EEE5F2E0DF012F
:1027C0001D928A95E9F785E00E943C140C94FA0367
:1027D000EF92FF920F931F93CF93DF93CDB7DEB7A6
:1027E0002A970FB6F894DEBF0FBECDBF8E010F5FE4
:1027F0001F4F8AE0F80111928A95E9F7F12C6F2DAD
:10280000C8010E946013F394F5E0FF12F8CF4AE08C
:1028100050E0B8018EE592E00E94F32B7C0121E0AC
:10282000892B09F420E0E114F10441F08AE0F80179
:10283000AEE5B2E001900D928A95E1F760917202E7
:1028400070E068597D4F45E08EE592E00E943D14AE
:10285000EF2819F40E94C31202C081E090E02A968A
:102860000FB6F894DEBF0FBECDBFDF91CF911F91A1
:102870000F91FF90EF9008950895FF920F931F938B
:10288000CF93DF938C01F62ED72FC42F222349F04C
:1028900081E08093F9010E9476249093F80180935F
:1028A000F7018091F9018823C1F08091F70190919F
:1028B000F8010E948E24059780F0EF2DFD2FD8019E
:1028C0004C2F50E0CD01801B910B841795071CF411
:1028D0008D918193F7CF1092F901DF91CF911F91E4
:1028E0000F91FF90089552985A9889B182FB8827DA
:1028F00080F908958091FC0181110DC00E94AB2BDD
:10290000811102C082E001C081E08093FC0182302D
:1029100011F40E94A62B81E09091FC01913009F006
:1029200080E008950E947314809304018091040153
:1029300061E0882311F080E001C081E00E94431A29
:102940000E947A1481110C94EC1408950E947A1458
:10295000811102C00C94EE14089581E09091FD0164
:102960009A3008F080E008950F931F93CF93DF9380
:10297000EC018B018091FD018A3038F4B801CE0161
:102980000E943C1581111DC00AC08091FA019091EE
:10299000FB010E948E24843F914080F715C08091F6
:1029A000FD018F3F19F08F5F8093FD018091FD0144
:1029B0008A3060F00E9476249093FB018093FA01A4
:1029C00003C01092FD0102C080E001C081E0DF91F0
:1029D000CF911F910F9108950C9412220C941522FF
:1029E000DF92EF92FF920F931F93CF93DF937901C2
:1029F000C82F880FDD0B41155105A9F0FE0193E0AA
:102A0000EE0FFF1F9A95E1F7EB5FFE4F81819281F8
:102A100082509E4F208130E04217530708F49A01FC
:102A2000A9010E94002CCE010E94FE22D82E8823EC
:102A3000D1F001151105B9F083E0CC0FDD1F8A95A7
:102A4000E1F7FE01EB5FFE4F438150E004171507ED
:102A500008F4A801CB5FDE4F6C817D8162507E4F10
:102A6000C7010E94002C8D2DDF91CF911F910F91F6
:102A7000FF90EF90DF9008950C94A3160C94C71666
:102A80000F931F93CF93DF9300D000D0CDB7DEB765
:102A900060911D0270911E0280911F029091200290
:102AA0000E949D24643671058105910528F10E94DC
:102AB0005E12DC01CB010296A11DB11D89839A83B0
:102AC000AB83BC8300E010E020E030E044E050E065
:102AD000BE016F5F7F4F82E00E94F014182F8823A1
:102AE00061F00E94822460931D0270931E02809305
:102AF0001F029093200201C011E0812F0F900F90D0
:102B00000F900F90DF91CF911F910F910895AF9289
:102B1000BF92CF92DF92EF92FF920F931F93CF93CA
:102B2000DF937C015B016A010E94AD14811103C037
:102B300001E010E002C00AE010E0C1E0D0E0F8944B
:102B4000B501C701F60109957894811115C0219648
:102B50000C171D0794F0CC9F9001CD9F300D300DC8
:102B6000112480E090E045E34A95F1F700000196DA
:102B700082179307C1F7E3CF81E0DF91CF911F91D7
:102B80000F91FF90EF90DF90CF90BF90AF9008959E
:102B90000F931F93CF93DF93CDB7DEB728970FB670
:102BA000F894DEBF0FBECDBFCE0101960E94481C37
:102BB00018856091210270912202809123029091E8
:102BC00024020E949D24643671058105910510F44C
:102BD0001123D9F000E010E020E030E048E050E0C0
:102BE000BE016F5F7F4F83E00E94F014882359F08D
:102BF0000E94822460932102709322028093230218
:102C00009093240202C080E003C00E94451C81E032
:102C100028960FB6F894DEBF0FBECDBFDF91CF91DF
:102C20001F910F910895AF92BF92CF92DF92EF92D2
:102C3000FF920F931F93CF93DF9300D000D000D06B
:102C4000CDB7DEB77B01C0904C01D0904D0101E0C3
:102C500010E09E012A5F3F4F40E050E060E070E0EE
:102C600080E00E94F014182F882309F43EC056011A
:102C70008FEFA81AB80A6091190270911A02809118
:102C80001B0290911C020E949D24643671058105EF
:102C9000910518F105E010E09E012F5F3F4F40E0E5
:102CA00050E060E070E081E00E94F014182F65E0D1
:102CB00070E0C5010E94621F91E02E81281390E010
:102CC000192339F10E9482246093190270931A0229
:102CD00080931B0290931C0211C065E070E0C50157
:102CE0000E94621F9E818913D5CF85E0F60131963F
:102CF000DE01119601900D928A95E1F7112349F0BA
:102D000085E0FE013196A4E1B2E001900D928A9532
:102D1000E1F785E0E4E1F2E0D70101900D928A95B8
:102D2000E1F7812F26960FB6F894DEBF0FBECDBF18
:102D3000DF91CF911F910F91FF90EF90DF90CF9097
:102D4000BF90AF9008950F931F93CF93DF93EC0143
:102D50008B0143E156E10E948715882391F040E4FE
:102D600055E1B801CE010E948715882351F048EC47
:102D700055E1B801CE01DF91CF911F910F910C94D5
:102D8000871580E0DF91CF911F910F9108950F93E8
:102D90001F93CF93DF93F894C0914C01D0914D01D4
:102DA000CE01019625E0FB01DC0101900D922A95F0
:102DB000E1F765E070E00E94621F88837894F894E0
:102DC0006E817F8188859985009110021091110292
:102DD0002091120230911302601771078207930746
:102DE00051F060931002709311028093120290933D
:102DF00013020E9441127894F8948989882331F053
:102E000060E0CE010A960E94201D198A7894DF9115
:102E1000CF911F910F9108950E946C260E94BC0FC4
:102E20000C9478260E947C260E9456100C949626BC
:102E30000E9461240E9453260E94AA0F0E940C1730
:102E40000E9412170E94B40FFBCF80912B0280FFCB
:102E500006C060912A0170E0660F771F26C081FFCF
:102E600004C060912A0184E005C082FF07C0609120
:102E70002A0188E0689FB001112417C090912A02AE
:102E80009923D1F060912901961788F720912A01A2
:102E900088E0289F90011124929FA001939F500DDC
:102EA000112470E0CA010E94CC2B6038710540F4F7
:102EB0006115710519F406C068E070E0862F089569
:102EC0008FE7089581E0089580912B0280FF08C06C
:102ED0006091260170E0759567957595679521C09D
:102EE00081FF06C06091260170E07595679519C055
:102EF00082FF04C06091260170E010C09091290209
:102F0000992399F0609125019617A0F780912601E9
:102F1000899FC001112470E00E94CC2B603871059C
:102F200040F46115710519F406C061E070E0862F68
:102F300008958FE7089581E008958D3E21F40E9461
:102F40002517819504C08E3E29F40E942517809391
:102F50002F0208958F3E21F40E942517819504C009
:102F6000803F29F40E94251780932E020895893FFF
:102F700019F40E94641705C08A3F31F40E94641757
:102F800081958093300208958B3F21F40E9464174D
:102F9000819504C08C3F29F40E946417809331020C
:102FA00008959FE0980F983078F421E030E0A9016F
:102FB00002C0440F551F9A95E2F7CA0190912D0265
:102FC000892B80932D0208958D3F21F480912B024F
:102FD00081600BC08E3F21F480912B02826005C07E
:102FE0008F3F29F480912B02846080932B020895F7
:102FF0008D3E39F490912F0297FF35C010922F0229
:1030000059C08E3E29F490912F021916BCF32BC0A3
:1030100090912E028F3E29F497FF25C010922E0228
:1030200049C0803F19F41916CCF31DC090913002AD
:10303000893F29F41916BCF4109230023BC08A3F34
:1030400019F497FF10C0F8CF8B3F39F490913102FB
:1030500097FF09C0109231022DC08C3F21F490914E
:1030600031021916BCF39FE0980F983080F421E0EC
:1030700030E0A90102C0440F551F9A95E2F7CA013A
:10308000809590912D02892380932D0213C08D3F4E
:1030900021F480912B028E7F0BC08E3F21F4809112
:1030A0002B028D7F05C08F3F29F480912B028B7FEF
:1030B00080932B0280912E02811106C080912F02F5
:1030C000811102C010922A0280913002811106C043
:1030D00080913102811102C01092290208950E944C
:1030E000762420912E02211104C020912F02222348
:1030F00021F0909328028093270220913002211121
:1031000004C020913102222321F090932602809363
:1031100025028CE292E00C94A123EF92FF920F9390
:103120001F93CF93DF9300D000D000D0CDB7DEB790
:1031300086E0ECE2F2E0DE01119601900D928A95B4
:10314000E1F7E0902E02F0902F02009130021091F2
:10315000310210922E0210922F0210923002109221
:103160003102E11003C0FF2009F45DC08091270205
:10317000909128020E948E24AC0190912A029923FA
:1031800039F020912B0130E02417350758F04BC05F
:1031900020912C018AE0289F9001112424173507E3
:1031A00018F041C09F3F19F09F5F90932A02EE20D4
:1031B00061F00E9425171E1414F09FEF01C091E0EA
:1031C000989F902D112490932E02FF2061F00E9471
:1031D00025171F1414F09FEF01C091E0989F902DC8
:1031E000112490932F0230912E023323E1F020918D
:1031F0002F022223C1F045EB3403C001112499238F
:1032000019F090932E0203C081E080932E0235EBDB
:103210002303C0011124992319F090932F0203C0B6
:1032200081E080932F02011103C0112309F45DC0D6
:1032300080912502909126020E948E24AC019091EB
:103240002902992339F02091270130E0241735070E
:1032500058F04BC0209128018AE0289F900111244A
:103260002417350718F041C09F3F19F09F5F9093D6
:103270002902002361F00E946417101614F09FEFDA
:1032800001C091E0989F902D11249093300211235A
:1032900061F00E946417111614F09FEF01C091E0D5
:1032A000989F902D11249093310230913002332356
:1032B000E1F0209131022223C1F045EB3403C0013B
:1032C0001124992319F09093300203C081E0809378
:1032D000300235EB2303C0011124992319F0909398
:1032E000310203C081E08093310280912E0281116E
:1032F0000BC080912F02811107C080913002811193
:1033000003C08091310281110E946F18EB82FC8210
:103310000D831E8386E0FE013196ACE2B2E001909F
:103320000D928A95E1F726960FB6F894DEBF0FBE90
:10333000CDBFDF91CF911F910F91FF90EF90089536
:10334000ECE2F2E086E0DF011D928A95E9F7109247
:103350002A021092290210922B020895EF92FF92F6
:103360000F931F93CF93DF938B01682F11110AC026
:10337000442329F0E82FF0E0E252FB4F6491762FCE
:10338000862F75C0212F30E0E82FF0E0442321F094
:10339000E252FB4FE491F0E046E0049FC0011124AB
:1033A000CFEFD0E0BE010E94B82B4BEA4603C0012C
:1033B000479F900D1124800F911D800F911D982F14
:1033C000990F890FAE01421B530B4E9FD0014F9FA7
:1033D000B00D5E9FB00D11249B2F189FA0011124EA
:1033E000452F55278E01041B150B0E9FA0010F9F23
:1033F000500D1E9F500D11247E01E81AF108E29E27
:103400008001E39E100DF29E100D1124212F332711
:10341000C21BD30BCE9F9001CF9F300DDE9F300D8E
:10342000112462307105A9F048F46115710569F045
:1034300061307105C9F48B2F752F0DC06430710593
:1034400081F058F06630710579F47E2F8B2F932F21
:103450000DC0832F7B2F9E2F09C08E2F7B2F952F82
:1034600005C08E2F732F02C07E2F852F692FDF910D
:10347000CF911F910F91FF90EF90089541E00E942E
:10348000AE1908950895EDE2F1E080836183089517
:103490000E943E1A0895CF93DF93762FE901682F9B
:1034A000842F0E94481A798368838A83DF91CF91A1
:1034B000089580917302282F269530E0211531055B
:1034C00019F48170826005C02F30310524F08170BD
:1034D0008C6180937302089588E090E00C94112C25
:1034E000CF92DF92EF92FF926B017C010E94591AFA
:1034F000B701A60188E090E0FF90EF90DF90CF90B9
:103500000C942F2CE3E7F2E083E0808311828FEFAD
:10351000828383831482ACE3B2E012968C9112977B
:10352000836012968C9360817181828193810C9467
:10353000701A8091730280FF02C08695089580E022
:10354000089590917702933018F49F5F90937702DB
:10355000882351F06091730270917402809175021A
:10356000909176020C94701A089581E00C94A11A3F
:1035700090917702992319F09150909377028823C4
:1035800051F0609173027091740280917502909174
:1035900076020C94701A089581E00C94B81A70E0C9
:1035A0000C94361F60912E018091730280FF0AC037
:1035B00080912D0123E0829FC001112488589D4FE6
:1035C0000C94CF1A80912F0190913001891780F7C8
:1035D000E82FF0E09F01220F331FE20FF31FE8589E
:1035E000FD4F1182108212828F5FF0CF9091730293
:1035F00090FF16C090912F0120913001921770F426
:10360000E92FF0E0DF01AA0FBB1FEA0FFB1FE8580C
:10361000FD4F8183608342839F5FF0CF0C94D21A69
:103620000895CF93DF9300D01F92CDB7DEB790916E
:10363000730290FF0AC09E012F5F3F4F0E944B1AFA
:103640004B8169818A810E94F61A0F900F900F902A
:10365000DF91CF910895CF93DF93EC01EC81F0E0FF
:10366000E256FC4F4491E3E7F2E0628181810E94DF
:10367000111B8C818F5F8C83DF91CF910895CF9345
:10368000DF93EC01E3E7F2E0438162818C810E94E9
:10369000111B8C818F5F8C83DF91CF910895EF9206
:1036A000FF920F931F93CF93DF9300D01F92CDB75C
:1036B000DEB7082FF62E142FE22E8091730280FFC2
:1036C00046C0E82FE695F0E0E25BFE4F90819093D4
:1036D0003C028E7F823061F49E012F5F3F4F802F2E
:1036E0000E944B1A4B8169818A810E94F61A0CC094
:1036F000923019F41091760207C0963019F40091B7
:10370000740202C09930D9F380917402081308C082
:1037100080917502F81204C080917602181729F082
:1037200080913E02826080933E0200937402F09288
:10373000750210937602EE2051F060917302709141
:10374000740280917502909176020E94701A0F9017
:103750000F900F90DF91CF911F910F91FF90EF90FD
:103760000895E3E7F2E09181282F4381628188E0A8
:10377000890F0C944F1B81E00C94B11BE3E7F2E03E
:103780009181282F4381628188EF890F0C944F1B10
:1037900081E00C94BE1BE3E7F2E0628128E0620F57
:1037A00008F46FEF282F438181810C944F1B81E037
:1037B0000C94CB1BE3E7F2E0628128E0621B08F483
:1037C00060E0282F438181810C944F1B81E00C9491
:1037D000DA1BE3E7F2E0438128E0420F08F44FEF01
:1037E000282F628181810C944F1B81E00C94E91B8E
:1037F000E3E7F2E0438128E0421B08F440E0282F91
:10380000628181810C944F1B81E00C94F81B20E0B5
:103810000C944F1BFF920F931F93CF93DF93EC01F8
:10382000F12C0FEF10E060913101F616F0F4809169
:103830002F012F2D30E0280F311DC901880F991F4E
:10384000280F391F28583D4F70E0C8010E94CC2B2B
:10385000962F8C814091760260917502F99E800DC1
:1038600011240E944B1AF394DECF0E94D21A9A813F
:103870008C8190FF02C08F5F01C081508C83DF91EB
:10388000CF911F910F91FF90089510923E020895DD
:1038900025E0E3E7F2E0DC0101900D922A95E1F7E3
:1038A00020913C0230913D0240913E02FC01258373
:1038B00036834783089560917302669570E041E016
:1038C00050E082E391E00E94E62B892B19F481E01D
:1038D00080933D020E9479129093360280933502C4
:1038E00080913E02846080933E020895ECE3F2E012
:1038F000118282818460828308959091730290FF87
:103900003AC09170811102C0926006C08F3010F0F1
:103910009C6102C0880F982B9093730280913E02A5
:10392000816080933E02662351F060917302709132
:10393000740280917502909176020E94701A6091D3
:103940007302669570E041E050E082E391E00E94EE
:10395000E62B892B19F00E94761C02C00E945B1C8A
:1039600081E08093380240917602609175028091E7
:1039700074020C94071C0895682F90917302969519
:1039800081E0890F8F3008F081E00C947D1C81E08C
:103990000C94BC1C682F9091730296958FEF890F41
:1039A00009F48EE00C947D1C81E00C94CA1C61E04B
:1039B0000C947D1CE3E7F2E0808181608083869532
:1039C0000C94D71C60E00C947D1CE3E7F2E080814E
:1039D0008E7F808360817181828193810E94701AC1
:1039E0000E94761CECE3F2E08281816082832FEFFB
:1039F00080E792E0215080409040E1F700C0000055
:103A00000C94D21A8091730280FD0C94E51C0C94E6
:103A1000DA1CE3E7F2E080818E7F80830E94761CCF
:103A2000ECE3F2E08281816082832FEF80E792E015
:103A3000215080409040E1F700C000000C94D21A61
:103A40001F93CF93DF93EC01162F8F8180FF0FC060
:103A5000888180FF0AC08091730281608093730225
:103A6000888186950E947D1C02C00E94091D8F815D
:103A700081FF06C0212F4B816A8189810E944F1BE3
:103A80008F8182FF08C08E81882319F00E945B1C01
:103A900002C00E94761C8F8183FF03C081E0809367
:103AA0003802DF91CF911F91089580913B028111DF
:103AB00033C00E94D20E811104C00E947A0F0E946E
:103AC000821A0E946C1A609373027093740280933E
:103AD00075029093760280913E02836080933E024D
:103AE0006E7F61F40E94821A0E946C1A60937302C6
:103AF0007093740280937502909376020E94591A13
:103B00000E94761C8091730280FF03C086950E94FC
:103B1000E21C81E080933B020895EF92FF920F93A5
:103B20001F93CF93DF9380913D02882309F47DC0DA
:103B300080913C02E0917302E695E81BE093370226
:103B4000823049F4F0E0E656FC4FE491CE2FD0E00D
:103B50000BE21BE11BC0863049F4F0E0E956FC4F54
:103B6000E491CE2FD0E00FE31BE110C0893051F477
:103B7000E695F0E0EC56FC4FE491CE2FD0E00AE061
:103B80001CE104C0C0EDD7E002E41AE180913802E4
:103B9000882361F0109238020E94791290933602C5
:103BA0008093350210923A02109239020E947912E3
:103BB000E0913502F09136029C012E1B3F0B2F3F06
:103BC0003F4798F5209134022223B1F0109234023D
:103BD0002091320230913302821B930B8F3F9F471B
:103BE00058F4205D3A48309333022093320280919A
:103BF0003E02886080933E02E0903902F0903A02E3
:103C0000CE0FDF1FD0933602C093350285E392E0DA
:103C1000F80109958091390290913A02892B29F493
:103C2000EF2819F081E080933402DF91CF911F914A
:103C30000F91FF90EF900895882311F0FA0101C0D1
:103C4000FB010994CF93DF93C82FD62F0E94991AB6
:103C50008C1740F00E94991A8D1720F4DF91CF91B4
:103C60000C94C71C8C2FDF91CF910C94D71C1F9301
:103C7000CF93DF93FB011281111196C0EC010E94DA
:103C8000EF0D8272CB3CFCE5DF0709F473C010F541
:103C9000C63CECE5DE0709F454C058F4C43C9CE58E
:103CA000D90709F442C008F045C0C33CDC45D1F156
:103CB00037C0C83C9CE5D90709F44DC008F446C09C
:103CC000C93CFCE5DF0709F44BC0CA3CDC4509F4FC
:103CD0004CC026C0C03DECE5DE0709F461C088F4A5
:103CE000CD3C9CE5D90709F44FC008F448C0CE3C50
:103CF000FCE5DF0709F44DC0CF3CDC4509F44DC0BD
:103D00000FC0C73D9CE5D90738F4C23DDC4508F03B
:103D10004BC06EE089E046C0CE35DD4509F444C0B5
:103D200011E042C00E94021D3FC044ED5CE167EC1F
:103D30007CE104C047EC5CE164ED7CE10E941C1E68
:103D400033C048EC5BE16BEB7BE1F8CF4BEB5BE125
:103D500068EC7BE1F3CF46EE5BE167ED7BE1EECF14
:103D600047ED5BE166EE7BE1E9CF44E05CE165EFC6
:103D70007BE1E4CF45EF5BE164E07CE1DFCF4CEC3D
:103D80005AE165EB7AE1DACF45EB5AE16CEC7AE186
:103D9000D5CF81E00E94D71C07C065E082E002C059
:103DA00068E086E00E94221E812FDF91CF911F9153
:103DB0000895E1E8F0E080818860808380818160FF
:103DC00080838FB7F89420ED33E0309389002093FF
:103DD00088008FBF0895EFE6F0E0808182608083E5
:103DE0000895EFE6F0E080818D7F808308951F9233
:103DF0000F920FB60F9211242F933F934F935F931F
:103E00006F937F938F939F93AF93BF93EF93FF93A2
:103E100080913F02909140020196909340028093DE
:103E20003F02811103C082E00E947504E0914002CC
:103E3000E695E695F0E0E256FB4FE49180913F0273
:103E40008E1303C080E00E947504FF91EF91BF9133
:103E5000AF919F918F917F916F915F914F913F9122
:103E60002F910F900FBE0F901F901895539A2BB162
:103E7000277F3BB138604FB7F894FC01CB01880F26
:103E8000991F680F791F6E0F7F1FE617F70789F0DC
:103E9000819198E03BB9000000C087FF2BB9880FE3
:103EA000000000C000C000C02BB900C09A9591F777
:103EB000ECCF4FBF8FE594E00197F1F700C0000011
:103EC00008950895FC01680F791F8FEF91E3E617BD
:103ED000F70771F02191822728E030E087FF03C0C7
:103EE000880F892701C0880F21503109B9F7EFCF1A
:103EF0000895CF93DF93EC01FB018281882309F4BD
:103F00003CC1C430FDE5DF0760F4CB3F9CE5D90739
:103F100088F49E0122503C452431310508F02EC121
:103F200009C0C236EDE5DE0729F0C63AFDE5DF0738
:103F300009F024C10E94E50E90935C0280935B021D
:103F4000C1318CE5D80709F4C6C008F042C0C930B9
:103F5000ECE5DE0709F49BC000F5C5308CE5D80719
:103F600009F485C078F4C330ECE5DE0709F478C0C5
:103F700008F07AC0C230DC4509F0F5C080915B02E0
:103F80008160EFC0C7309CE5D90709F478C008F01C
:103F90007AC080915B028061E4C0CD30FCE5DF0730
:103FA00009F487C058F4CB309CE5D90709F479C0EF
:103FB00008F07BC080915B0288606FC0CF30FCE569
:103FC000DF0709F480C008F082C080915B02877F20
:103FD000C8C0CE3F9CE5D90709F471C000F5C531D2
:103FE000FCE5DF0709F485C068F4C3319CE5D90717
:103FF00009F475C008F095C00E946C0880915B02BE
:104000008F77AFC0CC3FFCE5DF07A9F108F054C0C3
:10401000CB3FDC4509F0A7C080915C0240C0C230B4
:10402000EDE5DE0709F489C058F4C1158DE5D80720
:1040300009F45AC008F069C080915C0282602FC008
:10404000C236EDE5DE0709F47CC0C63AFDE5DF07C0
:1040500009F481C0C330DD4509F085C080E06EC041
:1040600080915B0282607DC080915B0216C080916E
:104070005B02886076C080915C0282604FC0809154
:104080005B0280626EC080915B0280646AC00E94A5
:104090006C0880915B02806864C0846062C081604B
:1040A0003DC080915B028E7F5CC080915B028D7F02
:1040B00058C080915B0216C080915C0218C080914C
:1040C0005C028D7F2BC080915B028F7E4AC0809105
:1040D0005B028F7D46C080915B028F7B42C08091E6
:1040E0005B02877F8B7F3DC080915C028D7F8E7FDE
:1040F00015C080915B0282FB222720F991E0922774
:1041000090FB82F990FB83F92CC080915C02982F80
:10411000909591708E7F892B90FB81F980935C0242
:1041200022C00E946C0880915B0287FB222720F945
:1041300091E0922790FB87F914C081E00E947C0FE8
:1041400012C080915B0284FB222720F991E0922724
:1041500090FB84F906C080915B02982F909590FBAC
:1041600080F980935B0280915B0290915C020E94D7
:10417000F60E0E946C0880E001C081E0DF91CF91D3
:104180000895CF93DF9386319C4541F5EB010E9462
:10419000EF0D982F8A81209102013091030188232D
:1041A00079F09A7A81E009F480E0809341029111DC
:1041B00002C069E201C065E3C9010E941D240AC072
:1041C00080914102811102C069E201C065E3C90129
:1041D0000E941F240E94310E80E001C081E0DF9127
:1041E000CF9108950F931F93CF93DF93C42FD22FB6
:1041F000FC0182818823C9F0409344020E94762406
:10420000909343028093420280E28C0F883008F042
:1042100057C0C77081E001C0880FCA95EAF7DF91E7
:10422000CF911F910F910C94F50580914402481392
:1042300030C080914202909143020E948E24883CBB
:10424000910538F510E21D0FCD17B9F080E28C0F03
:10425000883040F4C77081E001C0880FCA95EAF742
:104260000E94FC05183028F581E09D2F977001C051
:10427000880F9A95EAF70E94F505802F0E94EC05B9
:104280001830F0F4D77081E001C0880FDA95EAF7B2
:104290000AC080E28C0F883098F4C77081E001C0BA
:1042A000880FCA95EAF7DF91CF911F910F910C9477
:1042B000FC05802FDF91CF911F910F910C94EC059D
:1042C000DF91CF911F910F9108950F939C01CB0126
:1042D000243F4CE5340731F188F4293DFCE53F07E4
:1042E000D9F02A3D4CE5340779F1283D3C45A9F544
:1042F00006E221EE41EE68ED7CE52BC0263FFCE5B1
:104300003F07E1F0A8F0273F3C4539F507E225EEED
:1043100046EE67EF7CE51DC007E225EE45EE69ED50
:104320007CE517C006E221EE40EE64EF7CE511C0AB
:1043300007E225EE44EE65EF7CE50BC006E221EED8
:1043400042EE66EF7CE505C008E221E045EE6AED4D
:104350007CE50E94F22080E008C0FC018281882375
:1043600019F01092440201C081E00F9108958EE18E
:10437000489B02C08150E1F7489BFECF08955898B2
:1043800080E28A95F1F7589A0895FC012AE02A956F
:10439000F1F728E090E080E031E040E14A95F1F764
:1043A000880F489B02C08160932700C0000040E155
:1043B0004A95F1F7215089F720E12A95F1F729B1C3
:1043C00000C0000030E13A95F1F72170922720817A
:1043D000920F90830895EF92FF920F931F93CF93C4
:1043E000DF931F92CDB7DEB719828C017C01E60EF8
:1043F000F11C0E151F0551F00E94B721CE01019648
:104400000E94C521F80181938F01F3CF81E099814A
:10441000911180E00F90DF91CF911F910F91FF904C
:10442000EF900895509A589A08955098589AE89A9B
:10443000E9E6F0E080818C7F80830895615091E00F
:1044400001C0990F6A95EAF720E031E0992361F005
:10445000492F482319F0589A232701C0589840E261
:104460004A95F1F79695F2CF222311F0589A01C0A0
:10447000589880E28A95F1F758980895FF920F9323
:104480001F93CF93DF93EC018C01060F111DC01712
:10449000D10741F0F9900E94BF2168E08F2D0E9462
:1044A0001E22F5CFDF91CF911F910F91FF900895BC
:1044B0001F920F920FB60F9211240F931F932F93F9
:1044C0003F934F935F936F937F938F939F93AF939C
:1044D000BF93EF93FF93CF93DF931F92CDB7DEB7D8
:1044E00019820E94B721CE0101960E94C521082F92
:1044F000069506950695902F96959570202F257018
:10450000920F292F237096959695920F8770891395
:104510005FC0898181115CC0053008F059C080E11D
:104520008A95F1F7589A509A82E08A95F1F700C07F
:10453000589888E0089F80011124D801AB5FBE4FD6
:104540001696ED91FC9117973097A9F060914C0168
:1045500070914D0114962D913C911597260F371FA0
:1045600011968D919C911297680F791F13964C911B
:1045700013978C910995F801EB5FFE4F63816623D9
:1045800051F080914C0190914D0124813581820F31
:10459000931F0E943E220E94BF2180E18A95F1F77D
:1045A00058985098589A80E18A95F1F7F801EB5F96
:1045B000FE4F6081662351F080914C0190914D0136
:1045C00021813281820F931F0E94EB210E94B7212B
:1045D0000F90DF91CF91FF91EF91BF91AF919F919C
:1045E0008F917F916F915F914F913F912F911F918B
:1045F0000F910F900FBE0F901F9018950F931F9360
:10460000CF93DF93853091050CF06DC0EC01F894E9
:10461000509A589885E08A95F1F700009C2F96955E
:1046200095702C2F2570920F892F837096959695F3
:1046300023E0CC0FDD1F2A95E1F7980F8E01092B9F
:104640000E94BF2184E08A95F1F700C068E0802FC6
:104650000E941E2280E18A95F1F75098589A489955
:1046600002C000C0FCCF87E090E0489B08C00197E3
:1046700021F4509A589A789436C000C0F6CFFE01C3
:10468000EB5FFE4F6381662381F080914C01909136
:104690004D0124813581820F931F0E94EB218111EE
:1046A00004C0509A589A78941FC00E94B72180E2A3
:1046B0008A95F1F75898509A80E18A95F1F7CB5F87
:1046C000DE4F6881662351F080914C0190914D013D
:1046D00029813A81820F931F0E943E220E94BF21AE
:1046E000789481E001C080E0DF91CF911F910F911C
:1046F000089590935F0180935E01089590934B021B
:1047000080934A0208950E947A14811103C0809117
:1047100045020895E0914A02F0914B02309721F052
:104720000190F081E02D099480E00895E0914A0223
:10473000F0914B02309721F00280F381E02D099433
:104740000895E0914A02F0914B02309739F022E04F
:10475000DC012C930480F581E02D099408952091CB
:104760004802309149022817390771F090934902A5
:1047700080934802E0914A02F0914B02309721F079
:104780000680F781E02D099408952091460230912A
:1047900047022817390771F0909347028093460229
:1047A000E0914A02F0914B02309721F00084F185AC
:1047B000E02D09940895FC01329697E080E0915035
:1047C00029F021912223D9F38F5FF9CF0895662331
:1047D00049F0FC01329608962191621729F0E817FA
:1047E000F907D1F780E0089581E008959C01FC016C
:1047F00032969FEF80E04191461789F09F3F19F470
:10480000411101C0982F8F5F8630A9F79F3F39F083
:10481000F901E90FF11D97FDFA9562830895089556
:104820009C012A5F3F4FFC014281461301C0128266
:10483000019682179307B9F708950C94F6230C9408
:104840001024029626E0FC0111922A95E9F70895BA
:1048500008950C94282483E080934C020C9429241E
:10486000811102C081E001C082E080934C020C946F
:1048700029240C94302481E080934C020C94292448
:104880000C943B2408950C9442240C9443240C94DF
:1048900042240C9442240C944224CF930E94492435
:1048A0000E94E8130E944724C0E08C2F0E94A912A6
:1048B000811104C0CF5FCA30C1F701C081E0CF9140
:1048C0000895089580918602843011F00C94670455
:1048D00008950E946C080C94690482E084BD93E002
:1048E00095BD9AEF97BD80936E0008952FB7F89409
:1048F00080917E0290917F02A0918002B09181020E
:104900002FBF08952FB7F89460917E0270917F02B7
:1049100080918002909181022FBF08959C014FB732
:10492000F89480917E0290917F02A0918002B091D4
:1049300081024FBF821B930B0895CF92DF92EF92BB
:10494000FF922FB7F894C0907E02D0907F02E09043
:104950008002F09081022FBFA7019601261B370B22
:10496000480B590BCA01B901FF90EF90DF90CF902F
:10497000089578941F920F920FB60F9211248F937F
:104980009F93AF93BF9380917E0290917F02A091FD
:104990008002B09181020196A11DB11D80937E021B
:1049A00090937F02A0938002B0938102BF91AF9158
:1049B0009F918F910F900FBE0F901F90189581E0DF
:1049C0008093E00080E28093D8001092C9008FE1CC
:1049D0009EE40197F1F700C0000087E090EBDC0156
:1049E00080938F0290939002A0939102B0939202D1
:1049F0009CE088E10FB6F894A895809360000FBE04
:104A000090936000FFCF8091550208950895089516
:104A100022E02093E9002FEF3091E800215035FD8E
:104A200006C035ED3A95F1F700002111F5CF209140
:104A3000E80025FF0BC040E050E066E070E00E9417
:104A400008278091E8008E778093E8000895CF933F
:104A5000DF9321E02093E9002FEF3091E80021500F
:104A600035FD06C035ED3A95F1F700002111F5CF7F
:104A70002091E80025FF14C0EC0140E050E068E020
:104A800070E00E9408278091E8008E778093E8000C
:104A900088E0FE01ADE4B2E001900D928A95E1F765
:104AA000DF91CF910895089580918502811109C009
:104AB0000E9499280E94F6288091E20084608093E9
:104AC000E20008951092850208950C9440246091AC
:104AD000820281E0611101C080E00E942B240C94CD
:104AE000EB1E9091860281E0943009F080E06091A5
:104AF00082020E9430240E94F11E0E9483230C94A3
:104B0000750442E061EC81E00E94122842E261EC0F
:104B100082E00E9412289091860281E0943009F090
:104B200080E0609182020C94392480918802833065
:104B300009F461C030F4813071F0823009F49AC018
:104B400008958A3009F486C08B3009F46CC089302E
:104B500009F0A8C020C080918702813A09F0A2C064
:104B60008091E800877F8093E80080918B0290918C
:104B70008C02892B21F468E08DE492E003C060E0B0
:104B800080E090E070E00E9453278091E8008B77EE
:104B90008093E800089580918702813209F082C0F5
:104BA00080918B0290918C02029708F07BC08091DB
:104BB000E800877F8093E8008091E80082FD05C0CF
:104BC000809186028111F8CF6DC02091F300809111
:104BD000F20090E0922B029731F48091F100813045
:104BE00011F0863021F48091F1008093550280917C
:104BF000E8008B7753C080918702813A09F052C058
:104C000080918B0290918C02892B09F04BC080918E
:104C1000E800877F8093E8008091E80080FFFCCF68
:104C200080913F0136C0809187028132D9F5809111
:104C30008B0290918C02892BA9F58091E800877FE7
:104C40008093E8000E9447288091890280933F0169
:104C50000C946C0880918702813221F58091E800E4
:104C6000877F8093E8000E94472880918A02809382
:104C70005602089580918702813AA1F48091E8005C
:104C8000877F8093E8008091E80080FFFCCF8091CF
:104C900056028093F1008091E8008E778093E800BF
:104CA0000C944728089584B7877F84BF0FB6F89483
:104CB000A8958091600088618093600010926000E8
:104CC0000FBE90E080E80FB6F89480936100909357
:104CD00061000FBE0C943B240E9499280E94F62884
:104CE000E2EEF0E080818460808378940C948B2BDA
:104CF00083E391E00C947E23809186028530A9F4B1
:104D000080918602853079F40E9462248091840229
:104D10008823B1F30E944D24882391F30E94F22648
:104D20000E946C08EDCF0C946924089508950C94AA
:104D30009926292F332723303105C9F060F421301B
:104D4000310581F02230310509F044C08BE390E059
:104D500026E036E043C021323105E1F02232310550
:104D600049F138C082E190E021E436E037C099276C
:104D70008130910549F028F0029761F5EEEDF5E0FC
:104D800005C0E2E0F6E002C0EEEEF5E0849190E0CE
:104D90009F0124C06115710541F061307105D1F4A6
:104DA00089E090E021E336E019C089E090E028E155
:104DB00036E014C06115710541F06130710551F4A0
:104DC00089E490E023E536E009C080E490E02CE936
:104DD00036E004C080E090E020E030E0FA0131836A
:104DE0002083089580E189BD82E189BD09B400FE78
:104DF000FDCF8091D8008F7D8093D8008091E00016
:104E000082608093E0008091E00081FDFCCF0895F6
:104E1000CF92DF92EF92FF920F931F93CF93DF9386
:104E2000EC018B017A010E946628811133C0E114E4
:104E3000F10439F0F70180819181081B190BC80F2B
:104E4000D91FC12CD12C0115110519F18091E80051
:104E500085FD16C08091E8008E778093E800E1140C
:104E6000F10449F0F70180819181C80ED91ED182E9
:104E7000C08285E00FC00E946628882321F30AC003
:104E800089918093F10001501109FFEFCF1ADF0AD9
:104E9000DACF80E0DF91CF911F910F91FF90EF90DB
:104EA000DF90CF90089520918D0230918E022617C9
:104EB000370748F06115710539F42091E8002E7725
:104EC0002093E80001C0B901FC0120E061157105E3
:104ED00079F1809186028823F1F18530F1F180919A
:104EE000E80083FD3CC08091E80082FD2EC08091E7
:104EF000E80080FFEBCF2091F3008091F20090E07A
:104F0000922B6115710551F08830910538F421918B
:104F10002093F100615071090196F3CF21E00897C9
:104F200009F020E08091E8008E778093E800CECFF2
:104F30002111CFCF0AC080918602882361F085308D
:104F400061F08091E80083FD0AC08091E80082FF53
:104F5000F2CF80E0089582E0089583E0089581E033
:104F6000089520918D0230918E022617370748F060
:104F70006115710539F42091E8002E772093E8003F
:104F800001C0B901FC0120E06115710591F180912A
:104F90008602882309F440C0853009F43FC080911F
:104FA000E80083FD3DC08091E80082FD2FC0809124
:104FB000E80080FFE9CF2091F3008091F20090E0BB
:104FC000922B6115710559F08830910540F42491B8
:104FD0002093F1003196615071090196F2CF21E0E2
:104FE000089709F020E08091E8008E778093E80030
:104FF000CBCF2111CCCF0AC080918602882361F0EB
:10500000853061F08091E80083FD0AC08091E8005E
:1050100082FFF2CF80E0089582E0089583E0089552
:1050200081E00895982F973068F59093E9009817DC
:1050300039F07091EC002091ED005091F00003C028
:10504000242F762F50E021FD02C09F5FECCF3091DE
:10505000EB003E7F3093EB003091ED003D7F3093CD
:10506000ED003091EB0031603093EB007093EC0079
:105070002093ED005093F0002091EE0027FDE5CF46
:1050800080E008958F708093E90081E00895809119
:10509000870287FF11C08091E80082FD05C08091E2
:1050A00086028111F8CF11C08091E8008B770BC088
:1050B00080918602882349F08091E80080FFF8CF34
:1050C0008091E8008E778093E80008952091E400B5
:1050D0003091E50095E64091EC00842F817040FF0F
:1050E00023C08091E80080FD1DC080918602882346
:1050F00099F0853099F08091EB0085FD11C04091C9
:10510000E4005091E5002417350729F3915011F080
:105110009A01E1CF84E0089582E0089583E0089544
:1051200081E0089580E008954091E80042FFDDCFDE
:1051300008950E9407290E940F29E0EEF0E0808187
:1051400081608083E8EDF0E080818F77808319BCF7
:10515000A7EDB0E08C918E7F8C9380818F7E8083D1
:105160001092850208950F931F93CF93DF930E94AF
:1051700007290E940F29C8EDD0E088818F778883A6
:1051800088818068888388818F7D888319BC10928C
:10519000860210928202109284021092830200EE24
:1051A00010E0F80180818B7F808388818160888313
:1051B00042E060E080E00E941228E1EEF0E08081B1
:1051C0008E7F8083E2EEF0E0808181608083808149
:1051D00088608083F80180818E7F808388818061F0
:1051E0008883DF91CF911F910F910895E8EDF0E052
:1051F00080818F7E8083E7EDF0E080818160808315
:1052000084E082BF81E0809385020C94B328E8EDAE
:10521000F0E080818E7F80831092E20008951092EA
:10522000DA001092E10008951F920F920FB60F92CC
:1052300011242F933F934F935F936F937F938F939B
:105240009F93AF93BF93EF93FF938091E10082FF11
:105250000BC08091E20082FF07C08091E1008B7F4C
:105260008093E1000E948A2B8091DA0080FF1FC0AA
:105270008091D80080FF1BC08091DA008E7F8093E0
:10528000DA008091D90080FF0DC080E189BD82E104
:1052900089BD09B400FEFDCF81E0809386020E94A3
:1052A000542505C019BC109286020E946225809187
:1052B000E10080FF19C08091E20080FF15C080915D
:1052C000E2008E7F8093E2008091E2008061809313
:1052D000E2008091D80080628093D80019BC85E0FC
:1052E000809386020E9467258091E10084FF30C090
:1052F0008091E20084FF2CC080E189BD82E189BDFC
:1053000009B400FEFDCF8091D8008F7D8093D80036
:105310008091E1008F7E8093E1008091E2008F7E9A
:105320008093E2008091E20081608093E2008091AE
:105330008202882311F084E007C08091E30087FD9A
:1053400002C081E001C083E0809386020E94712543
:105350008091E10083FF29C08091E20083FF25C096
:105360008091E100877F8093E10082E08093860254
:10537000109282028091E1008E7F8093E100809103
:10538000E2008E7F8093E2008091E2008061809352
:10539000E20042E060E080E00E9412288091F0008C
:1053A00088608093F0000E946525FF91EF91BF9186
:1053B000AF919F918F917F916F915F914F913F91AD
:1053C0002F910F900FBE0F901F9018951F920F9264
:1053D0000FB60F9211242F933F934F935F936F93C8
:1053E0007F938F939F93AF93BF93CF93DF93EF936D
:1053F000FF93C091E900CF708091EC00D82FD1705D
:1054000080FDD0E81092E9008091F000877F8093C2
:10541000F00078940E942A2A1092E9008091F0000E
:1054200088608093F000CD2BCF70C093E900FF918E
:10543000EF91DF91CF91BF91AF919F918F917F912C
:105440006F915F914F913F912F910F900FBE0F90F1
:105450001F9018951F93CF93DF93CDB7DEB7AA9710
:105460000FB6F894DEBF0FBECDBFE7E8F2E0809143
:10547000F100819322E0EF38F207C9F70E949525E9
:105480008091E80083FF2EC180918702909188026D
:10549000492F50E04A30510508F024C1FA01EE5975
:1054A000FF4F0C94E02B803821F0823809F01AC1AC
:1054B00008C08091830290918402992389F08260D0
:1054C0000FC080918B028F70873008F00BC18093E2
:1054D000E9008091EB0085FB882780F91092E900B4
:1054E0009091E800977F9093E8008093F1001092EC
:1054F000F100D1C0282F2D7F09F0F4C0882319F0C6
:10550000823061F0EFC080918902813009F0EAC0F9
:10551000933009F080E0809384022EC0809189024C
:1055200081112AC080918B028F702FEF280F2630B7
:1055300008F0D8C08093E9002091EB0020FF1CC048
:10554000933021F48091EB00806214C09091EB00C5
:1055500090619093EB0021E030E0A90102C0440F7C
:10556000551F8A95E2F74093EA001092EA00809175
:10557000EB0088608093EB001092E9008091E800D6
:10558000877F8093E8000E944728ACC08111AAC0A1
:10559000109189021F778091E3008078812B80939E
:1055A000E3008091E800877F8093E8000E9447280D
:1055B0008091E80080FFFCCF8091E30080688093B9
:1055C000E300111102C082E001C083E080938602F3
:1055D00089C08058823008F085C0809189029091FE
:1055E0008A028C3D53E0950779F583E08A838AE24D
:1055F00089834FB7F894DE01139620E03EE051E234
:10560000E32FF0E050935700E49120FF03C0E295B0
:10561000EF703F5FEF708E2F90E0EA3010F0C7968A
:1056200001C0C0968D939D932F5F243149F74FBFE2
:105630008091E800877F8093E8006AE270E0CE0105
:1056400001960E94532716C060918B0270918C02C4
:10565000AE014F5F5F4F0E949726BC01892B09F472
:1056600041C09091E800977F9093E80089819A81EA
:105670000E94B1278091E8008B778093E80032C0C8
:10568000803881F58091E800877F8093E8008091E1
:1056900082028093F1008091E8008E7772CF8111B1
:1056A00021C08091890290918A0299270297D4F4AF
:1056B0008091E800877F8093E80080918902809341
:1056C00082020E94472880918202811106C0809147
:1056D000E30087FD02C081E001C084E08093860280
:1056E0000E9481258091E80083FF0AC08091E80034
:1056F000877F8093E8008091EB0080628093EB00CD
:10570000AA960FB6F894DEBF0FBECDBFDF91CF9142
:105710001F9108950895CF93809186028823A1F068
:10572000C091E900CF709091EC00892F817090FDBD
:1057300080E8C82B1092E9008091E80083FD0E9468
:105740002A2ACF70C093E900CF9108950E9499282A
:10575000109286020895E8EDF0E0808180618083F8
:105760008AE18A95F1F700C08091D900817008958F
:10577000AA1BBB1B51E107C0AA1FBB1FA617B70777
:1057800010F0A61BB70B881F991F5A95A9F7809593
:105790009095BC01CD01089597FB072E16F4009457
:1057A00007D077FD09D00E94B82B07FC05D03EF446
:1057B000909581959F4F0895709561957F4F0895BD
:1057C000EE0FFF1F0590F491E02D0994FC0141506C
:1057D000504030F001900616D1F73197CF0108956F
:1057E000882799270895FB01DC0104C08D91019061
:1057F000801921F441505040C8F7881B990B089537
:10580000FB01DC0102C001900D9241505040D8F7DD
:105810000895F999FECF92BD81BDF89A992780B578
:105820000895A6E1B0E044E050E00C94432CA8E1D8
:10583000B0E042E050E00C94432C262FF999FECFC3
:1058400092BD81BDF89A019700B4021639F01FBAD3
:1058500020BD0FB6F894FA9AF99A0FBE08950396F0
:10586000272F0E941E2C0E941D2C252F0E941E2CCB
:10587000242F0C941E2C0196272F0E941E2C0C9472
:105880001D2CDC01CB01FC01F999FECF06C0F2BD55
:10589000E1BDF89A319600B40D9241505040B8F7EE
:0658A0000895F894FFCF0B
:1058A600C800D9010100000001000000000000004E
:1058B60005010000000406000000000000080A00C0
:1058C6000000000000280850011E0A140200020011
:1058D600020201032527250825532506250725014C
:1058E600F4F5F6F73133329497C63435FE010001EC
:0E58F600020202020606060909090909090054
:00000001FF
